:100000000C9465020C94A9020C94A9020C94A90208
:100010000C94A9020C94A9020C94A9020C94A902B4
:100020000C94A9020C94A9020C94B00B0C94820CB1
:100030000C94A9020C94A9020C94A9020C94A90294
:100040000C94A9020C940B210C94A9020C94A90203
:100050000C94A9020C94AD1A0C94A9020C94A90258
:100060000C94A9020C94A9020C94A9020C94A90264
:100070000C94A9020C94A9020C94A9020C94A90254
:100080000C94A9020C94A9020C94A9020C94A90244
:100090000C94A9020C94A9020C94A9020C94A90234
:1000A0000C94A9020C94A9020C94A902E70C090D66
:1000B000F40D090DF40D4B0D6E0DF40DC30DD60DA1
:1000C000C310C310F110F11033116F116F136F13C0
:1000D00087116F137E127E1249136F136F135D1316
:1000E0000000F0A135002B000152E100E00000000B
:1000F0001E00140004001D7100774E001F001A003E
:1001000016001B00007F4C002000080007000600BE
:10011000E2002A002100150009001900E3004B004D
:10012000220017000A00050000004A0029002F00E5
:1001300000002B0200004D002D00300000002B00BD
:100140000000500023001C000B00110000004F00B5
:10015000240018000D001000E700520025000C00DC
:100160000E003600E6002C00260012000F003700BB
:10017000007F2800270013003300387100775100FA
:100180002E0031823481E500E40000002900025293
:1001900001000100010000003A001E0220022202BC
:1001A000010051003B001F02210223020100280030
:1001B0003C002F0226022F0001002C003D003002DF
:1001C00027023000010052003E00240235003502B3
:1001D000000050000100360200002B0000004F001C
:1001E0000100370200002B0200004A003F003102EC
:1001F0003800310000004D0040005F005C005900F5
:1002000062004B00410060005D005A0037004C0066
:10021000420061005E005B0067002A00430054005A
:100220005500560057004E004400450001003900BB
:1002300058000000290002520100010001000000E6
:10024000A5000100010001000100B500A6000100A9
:10025000F200010001000100A800F000F100F1002F
:10026000F400B600AA00F900F3000100FA00B4009F
:10027000A9000100010001000000B8000100F90020
:100280000000FA000000B9000100F9000000FA00C7
:100290000000AC00010001004A0001000000AB00BA
:1002A0004600F9005000FA000100A9004B0052007E
:1002B000510051004E00AE00B30001004F0001009C
:1002C0000100AD00B10001004D0001000100AA00D5
:1002D00001000100010001000100000016034500BB
:1002E000720067006F0044006F0078002000450036
:1002F0005A00000016034500720067006F004400BA
:100300006F007800200045005A0000000403090433
:1003100009026D00040100A0FA09040000010301B4
:100320000100092111010001223F00070581030896
:10033000000A090401000103010200092111010062
:1003400001224D000705820308000A09040200018A
:100350000300000009211101000122360007058376
:100360000308000A09040300010300000009211129
:100370000100012239000705840310000112011059
:100380000100000008EDFE07130100010200010555
:10039000010906A101050719E029E71500250195C6
:1003A0000875018102050819012905950575019156
:1003B000029501750391010507190029771500259C
:1003C00001957875018102C005010980A1018502AE
:1003D00016010026B7001A01002AB7007510950112
:1003E0008100C0050C0901A1018503160100269CAE
:1003F000021A01002A9C02751095018100C00501B6
:100400000902A1010901A100050919012905150029
:10041000250195057501810295017503810105018D
:10042000093009311581257F950275088106093843
:100430001581257F950175088106050C0A3802157E
:1004400081257F950175088106C0C005010906A1B7
:1004500001050719E029E7150025019508750181B7
:100460000295017508810105081901290595057591
:100470000191029501750391010507190029FF15E6
:100480000025FF950675088100C0000000000000EF
:100490000000000000010204060A0F17202C3A4A4F
:1004A0005D71879DB3C7DAE9F5FCFFFCF5E9DAC7B2
:1004B000B39D87715D4A3A2C20170F0A060402018A
:1004C0000000000000000000000011241FBECFEF5C
:1004D000DAE0DEBFCDBF04B603FE24C08091EE019A
:1004E0009091EF01A091F001B091F1018730904B14
:1004F000A740B04BB9F41092EE011092EF011092A8
:10050000F0011092F10114BE84B7877F84BF88E1A7
:100510000FB6F89480936000109260000FBEE0E088
:10052000FFE3099511E0A0E0B1E0EAE9F5E402C0DB
:1005300005900D92A433B107D9F721E0A4E3B1E00F
:1005400001C01D92AE3EB207E1F70E94F6080C947E
:10055000CB220C94000061110BC0FC018281882326
:1005600021F085EE0E94570F03C085EE0E941F10F8
:1005700080E090E0089508956091B1017091B2011A
:100580008091B3019091B4010E94D91956985E9858
:1005900025982D9826982E9827982F98813019F015
:1005A000823021F00895259A2D9A0895269A2E9A40
:1005B00008950C94BC0256985E9825982D9826981C
:1005C0002E9827982F988FEF90E090938900809332
:1005D000880090938B0080938A0090938D00809385
:1005E0008C00259A2D9A2FEF80E792E021508040D1
:1005F0009040E1F700C00000269A2E9A2FEF80E786
:1006000092E0215080409040E1F700C00000279A1E
:100610002F9A2FEF80E792E0215080409040E1F741
:1006200000C0000025982D982FEF80E792E0215020
:1006300080409040E1F700C0000026982E982FEFF0
:1006400080E792E0215080409040E1F700C0000038
:1006500027982F9856985E9825982D9826982E982A
:1006600027982F98089589EA8093800089E08093E5
:10067000810024982C983F988AB18F748AB96E981B
:10068000479A8BB1806B8BB9769A0E94DB020C94EF
:10069000BB0280E2809300018091340181110EC081
:1006A0000E94980381E0809334012FEF83ED90E363
:1006B000215080409040E1F700C0000080E40E949B
:1006C0009E038093000181112EC00E94C803809375
:1006D0000001811128C00E94C8038093000181118C
:1006E00022C08FE30E94C8038093000181111BC0C8
:1006F0000E94C00380E40E949E0380930001811148
:1007000012C08CE00E94C8038093000181110BC0CD
:100710000E94C80380930001811105C08FE30E94ED
:10072000C803809300010E94C003809100010895D6
:100730001092B9008AE08093B800089594EA9093EB
:10074000BC009091BC0097FFFCCF9091B900987FBE
:10075000983021F0903111F081E008958093BB0032
:1007600084E88093BC008091BC0087FFFCCF80911F
:10077000B900887F883111F0803471F780E00895E6
:1007800084E98093BC008091BC0084FDFCCF089577
:100790008093BB0084E88093BC008091BC0087FFFD
:1007A000FCCF9091B900987F81E0983209F480E005
:1007B000089584E88093BC008091BC0087FFFCCF43
:1007C0008091BB00089580910001811115C080E4E3
:1007D0000E949E038093000181110CC082E10E945F
:1007E000C80380930001811105C08FEF0E94C803E8
:1007F000809300010E94C00384B1807F84B985B1D9
:10080000807F85B98AB1837F8AB98BB1837F8BB9A9
:100810003E98469808950E944903809300010E94E3
:10082000E30380B38C7080BB81B3836F81BBE4E44E
:10083000F1E0A6E3B1E011921D9281E0E235F80704
:10084000D1F70C943303BF92CF92DF92EF92FF92D5
:100850000F931F93CF93DF9380910001882379F04A
:10086000809135018F5F80933501811108C00E940E
:10087000490380930001811102C00E94DB0206E35C
:1008800011E0C0E0D0E0DD24D39482E0C82EEE2455
:10089000E394F12CC73000F580910001811162C012
:1008A00080E40E949E0380930001811112C082E1C6
:1008B0000E94C8038093000181110BC0C7010C2E58
:1008C00001C0880F0A94EAF780950E94C8038093BC
:1008D00000010E94C00346C0CA30A1F028F4C8300D
:1008E00059F0C93061F005C0CC3089F070F0CD30DE
:1008F00089F0209A289810C0219A29980DC0229A30
:100900002A980AC0239A2B9807C0529A01C0539A7A
:100910005B9802C03E9A4698E0EAEA95F1F78FB1FB
:1009200079995AC092E081708D25892B7C9B02C0F9
:1009300090E001C094E0892B7D9B02C090E001C053
:1009400098E0892B7E9B02C090E001C090E1892B4A
:100950009FB19095991F9927991F9295990F907E15
:10096000892B0FC08091000181114BC080E40E944F
:100970009E0380930001882389F1B12C0E94C0035B
:100980008B2DF8019081981719F08083C092010196
:100990000E94E30321960F5F1F4FCE30D10509F06F
:1009A00079CF80910101882371F1815080930101F9
:1009B000882339F08FE99FE00197F1F700C000002C
:1009C00022C0A4E4B1E0E6E3F1E081918D9391E0EF
:1009D000E434F907D1F717C090E0A5CF83E10E9476
:1009E000C803809300018111C8CF81E40E949E0357
:1009F000809300018111C1CF0E94D903B82EB09419
:100A0000BDCF80E0BECF0E94D90281E0DF91CF91BF
:100A10001F910F91FF90EF90DF90CF90BF900895BE
:100A2000E82FF0E0EC5BFE4F8081089508958B3B4A
:100A3000910578F4883A910540F5853A9105D0F40E
:100A40008430910508F0B1C08130910509F4ADC042
:100A50006BC0803E910508F467C0883E910508F49C
:100A6000A4C09C01205F31092031310508F05CC031
:100A700090650895853A910509F459C0863A910523
:100A800009F458C083E890E40895883A910509F480
:100A900054C0893A910509F453C08A3A910509F482
:100AA00052C08B3A910509F451C08C3A910509F472
:100AB00050C08D3A910509F44FC0803B910509F46F
:100AC0004EC08E3A910509F44DC08F3A910509F454
:100AD0004CC0813B910509F44BC0823B910509F460
:100AE0004AC0833B910509F449C0843B910509F450
:100AF00048C0853B910509F447C0863B910509F440
:100B000046C0873B910509F445C0883B910509F42F
:100B100044C0893B910509F443C08A3B910509F023
:100B200042C08AE296E4089580E090E0089581E86A
:100B300090E4089582E890E4089582EE94E40895A4
:100B400089EE94E408958AEE94E4089585EB94E4A4
:100B5000089586EB94E4089587EB94E408958CEC73
:100B600094E408958DEC94E4089583E895E4089561
:100B70008AE895E4089582E995E4089584E995E486
:100B8000089581E296E4089583E296E4089584E26C
:100B900096E4089585E296E4089586E296E4089541
:100BA00087E296E4089580E094E40895089596E03D
:100BB000799FF001112494E5899FE00DF11D112426
:100BC000E60FF11DEE0FFF1FEC51FF4F8591949141
:100BD0000895880F991F805A9040FC018591949147
:100BE0000895880F991F80529F4FFC018591949121
:100BF000089526E0729FF001112444E5849FE00DE2
:100C0000F11D1124E60FF11DEE0FFF1FEC51FF4FF8
:100C100025913491C9019A9581159F4110F4C9011C
:100C20000895C90190528115904128F4C9019F701F
:100C30000E94F1050895C90190538115904120F457
:100C4000C9019927906C0895211580E5380769F44A
:100C50000E9490139FEF24E34CE0915020404040CD
:100C6000E1F700C000000C94D21A213080E538076B
:100C700031F48091CC0181608093CC010895C90149
:100C800090558115904108F050C0832F99278F709F
:100C9000992781309105D9F4A9014370552702C0E5
:100CA000880F991F4A95E2F79C68A90164E0440FF8
:100CB000551F6A95E1F744275370842B952B73E0F9
:100CC000220F331F7A95E1F7207633271DC082303B
:100CD000910529F4922F8827816F906A08958330B7
:100CE0009105A9F4A9014370552781E090E002C065
:100CF000880F991F4A95E2F79C6843E0220F331F43
:100D00004A95E1F7207E3770822B932B0895049744
:100D1000F1F4A9014370552781E090E002C0880FEB
:100D2000991F4A95E2F79A68E8CFC9019057811553
:100D3000904120F4C9019F7090620895C9019058B4
:100D40008115904120F4C9019F70906A0895203E5A
:100D50003105E0F4203C310558F52133310509F423
:100D600070C048F42932310509F464C02A323105D3
:100D700009F46EC074C029333105F1F02238310511
:100D8000D9F02533310509F44EC069C0233E310541
:100D900089F138F4203E3105C1F0223E3105E1F001
:100DA0005EC0263E310569F1273E3105A9F157C0E5
:100DB000C9010E94E90508958091DF0180FD02C00C
:100DC00081FF4DC080EE90E04BC08091DF0180FF3D
:100DD000F9CF89E390E044C08091DF0182FF0EC02B
:100DE0008091DF0184FF03C080E090E039C083EE92
:100DF00090E036C08091DF0182FFF2CF82EE90E07A
:100E00002FC08091DF0183FF0BC08091DF0184FD43
:100E1000EBCF87EE90E024C08091DF0183FFF5CF18
:100E200086EE90E01DC08091DF0185FF07C089E25A
:100E300090E016C08091DF0185FFF9CF85E390E057
:100E40000FC08091DF0186FF07C08AE290E008C0F2
:100E50008091DF0186FFF9CF81E390E001C0C901F5
:100E60000E941705089508950C943307809162013C
:100E70000895CF93DF9300D01F92CDB7DEB72091B6
:100E8000E501243019F523E029839B838A8320938D
:100E9000E9008FEF9091E800815095FD06C095ED37
:100EA0009A95F1F700008111F5CF8091E80085FF58
:100EB0000DC040E050E063E070E0CE0101960E947A
:100EC000A3098091E8008E778093E8000F900F903F
:100ED0000F90DF91CF910895CF93DF9300D01F92B1
:100EE000CDB7DEB72091E501243021F522E029833A
:100EF0009B838A8383E08093E9008FEF9091E800E1
:100F0000815095FD06C095ED9A95F1F7000081118D
:100F1000F5CF8091E80085FF0DC040E050E063E030
:100F200070E0CE0101960E94A3098091E8008E77BF
:100F30008093E8000F900F900F90DF91CF9108956C
:100F40002091E5012430F1F422E02093E9002FEF15
:100F50003091E800215035FD06C035ED3A95F1F7A6
:100F600000002111F5CF2091E80025FF0BC040E0E3
:100F700050E065E070E00E94A3098091E8008E7760
:100F80008093E8000895CF93DF93EC018091E50111
:100F9000843009F046C090910C019923D9F09091CA
:100FA0000D019923B9F08093E9008FEF9091E8004B
:100FB000815095FD06C095E19A95F1F700008111E9
:100FC000F5CF8091E80085FF2CC040E050E060E163
:100FD00070E017C081E08093E9008FEF9091E80006
:100FE000815095FD06C095ED9A95F1F700008111AD
:100FF000F5CF8091E80085FF14C040E050E068E044
:1010000070E0CE010E94A3098091E8008E77809362
:10101000E80080E1FE01A2E5B1E001900D928A9521
:10102000E1F7DF91CF9108958091E401811109C02A
:101030000E94350B0E94920B8091E20084608093A5
:10104000E20008951092E401089508950C94F820A8
:101050000E94691A0E94FE200E942F0E0C943407F1
:1010600042E061EC81E00E94AF0A42E061EC82E084
:101070000E94AF0A42E061EC83E00E94AF0A42E1C5
:1010800061EC84E00C94AF0A8091E701833009F4AD
:1010900055C030F4813071F0823009F48EC008956B
:1010A0008A3009F47AC08B3009F460C0893009F0C5
:1010B0009CC020C08091E601813A09F096C08091E1
:1010C000E800877F8093E8008091EA019091EB012E
:1010D000892B21F060E080E090E003C060E182E5D0
:1010E00091E070E00E94EC098091E8008B7780939A
:1010F000E80008958091E601813209F076C0809180
:10110000EA019091EB01009719F0039709F06DC087
:101110008091E800877F8093E8008091E80082FD5D
:1011200005C08091E5018111F8CF5FC08091F10089
:10113000809362018091E8008B7753C08091E60133
:10114000813A09F052C08091EA019091EB01892B1C
:1011500009F04BC08091E800877F8093E800809180
:10116000E80080FFFCCF80910C0136C08091E60141
:101170008132D9F58091EA019091EB01892BA9F593
:101180008091E800877F8093E8000E94E40A8091C4
:10119000E80180930C010C9490138091E601813258
:1011A00021F58091E800877F8093E8000E94E40A9F
:1011B0008091E9018093630108958091E601813A6D
:1011C000A1F48091E800877F8093E8008091E80097
:1011D00080FFFCCF809163018093F1008091E80053
:1011E0008E778093E8000C94E40A089584B7877F93
:1011F00084BF88E10FB6F89480936000109260007D
:101200000FBE90E080E80FB6F89480936100909351
:1012100061000FBE0E947E0E0E94350B0E94920B51
:101220008091E20084608093E20078940E940D0E29
:101230000E94800E82E091E00E942A0E0E94E62029
:101240008091E501853069F40E942C1A8091E301B8
:101250008823B1F30E94541A882391F30E948D09C8
:10126000EFCF0E94860EECCF292F33272330310594
:10127000A9F06CF42130310509F442C02230310567
:1012800009F043C08DE690E020E133E042C0213216
:101290003105C9F02232310519F137C09927813063
:1012A000910541F08230910541F0892B71F5ECE018
:1012B000F3E005C0E4EFF2E002C0ECEDF2E084916F
:1012C00090E09F0126C0643000F5E62FF0E0EE0FBD
:1012D000FF1FEE5DFE4F2081318189E090E019C053
:1012E000643098F4E62FF0E0DF01AA0FBB1FA65E82
:1012F000BE4F2D913C91EA5EFE4F808190E009C087
:1013000082E190E02DE733E004C080E090E020E04F
:1013100030E0FA0131832083089580E189BD82E1C4
:1013200089BD09B400FEFDCF8091D8008F7D8093E8
:10133000D8008091E00082608093E0008091E0001E
:1013400081FDFCCF0895CF92DF92EF92FF920F9331
:101350001F93CF93DF937C018B01EA010E94050B61
:10136000811131C0209731F088819981081B190BB8
:10137000E80EF91EC12CD12C0115110519F180912F
:10138000E80085FD14C08091E8008E778093E80026
:10139000209741F0888199818C0D9D1D99838883C8
:1013A00085E011C00E94050B882331F30CC0F701C2
:1013B00081917F018093F10001501109FFEFCF1A55
:1013C000DF0ADACF80E0DF91CF911F910F91FF907C
:1013D000EF90DF90CF9008952091EC013091ED01D6
:1013E0002617370748F06115710539F42091E80098
:1013F0002E772093E80001C0B901FC0120E06115BF
:101400007105B9F18091E501882309F440C0853068
:1014100009F43FC08091E80083FD3DC08091E80061
:1014200082FF06C08091E80082FF26C080E0089518
:101430008091E80080FFE3CF2091F3008091F200DB
:1014400090E0922B6115710551F08830910538F4C8
:1014500021912093F100615071090196F3CF21E0B1
:10146000089709F020E08091E8008E778093E800EB
:10147000C6CF2111C7CFD6CF8091E501882339F09F
:10148000853039F08091E80083FFCCCF04C082E042
:10149000089583E0089581E008952091EC01309152
:1014A000ED012617370748F06115710539F42091D1
:1014B000E8002E772093E80001C0B901FC0120E08C
:1014C00061157105C1F18091E501882309F441C0DE
:1014D000853009F440C08091E80083FD3EC08091D2
:1014E000E80082FF06C08091E80082FF27C080E00C
:1014F00008958091E80080FFE3CF2091F300809170
:10150000F20090E0922B6115710559F08830910539
:1015100040F424912093F1003196615071090196B5
:10152000F2CF21E0089709F020E08091E8008E7763
:101530008093E800C5CF2111C6CFD5CF8091E501BA
:10154000882339F0853039F08091E80083FFCBCFD4
:1015500004C082E0089583E0089581E00895982F03
:10156000973058F59093E900981739F07091EC0096
:101570002091ED005091F00003C0242F762F50E011
:1015800021FF19C03091EB003E7F3093EB0030918A
:10159000ED003D7F3093ED003091EB0031603093F2
:1015A000EB007093EC002093ED005093F00020913D
:1015B000EE0027FF07C09F5FD3CF8F708093E900B5
:1015C00081E0089580E008958091E60187FD05C0DF
:1015D0008091E80080FF0EC012C08091E80082FD7B
:1015E00005C08091E5018111F8CF08958091E80050
:1015F0008B7708C08091E5018111EACF0895809131
:10160000E8008E778093E80008958091E40090913F
:10161000E50045E62091EC0020FF21C02091E80084
:1016200020FD21C02091E501222389F0253089F099
:101630002091EB0025FD0FC02091E4003091E500E2
:101640002817390739F3415041F0C901E3CF82E04F
:10165000089583E0089581E0089584E0089520913D
:10166000E80022FFDFCF80E008950E94A30B0E94D4
:10167000AB0BE0EEF0E0808181608083E8EDF0E08C
:1016800080818F77808319BCA7EDB0E08C918E7F2D
:101690008C9380818F7E80831092E40108950F9354
:1016A0001F93CF93DF930E94A30B0E94AB0BC8ED57
:1016B000D0E088818F77888388818068888388815B
:1016C0008F7D888319BC1092E5011092E101109280
:1016D000E3011092E20100EE10E0F80180818B7FBF
:1016E000808388818160888342E060E080E00E949E
:1016F000AF0AE1EEF0E080818E7F8083E2EEF0E0E1
:10170000808181608083808188608083F80180810E
:101710008E7F8083888180618883DF91CF911F9144
:101720000F910895E8EDF0E080818F7E8083E7EDF2
:10173000F0E080818160808384E082BF81E08093DB
:10174000E4010C944F0BE8EDF0E080818E7F808304
:101750001092E20008951092DA001092E1000895CC
:101760001F920F920FB60F9211242F933F934F9316
:101770005F936F937F938F939F93AF93BF93EF93F9
:10178000FF938091E10082FF0BC08091E20082FF15
:1017900007C08091E1008B7F8093E1000E940C0ED6
:1017A0008091DA0080FF1FC08091D80080FF1BC0AD
:1017B0008091DA008E7F8093DA008091D90080FFDB
:1017C0000DC080E189BD82E189BD09B400FEFDCF75
:1017D00081E08093E5010E94140805C019BC1092B5
:1017E000E5010E9422088091E10080FF19C08091EC
:1017F000E20080FF15C08091E2008E7F8093E200BE
:101800008091E20080618093E2008091D800806244
:101810008093D80019BC85E08093E5010E942608DA
:101820008091E10084FF30C08091E20084FF2CC0F1
:1018300080E189BD82E189BD09B400FEFDCF8091C0
:10184000D8008F7D8093D8008091E1008F7E8093B7
:10185000E1008091E2008F7E8093E2008091E200BF
:1018600081608093E2008091E101882311F084E09F
:1018700007C08091E30087FF02C083E001C081E0E0
:101880008093E5010E9428088091E10083FF29C030
:101890008091E20083FF25C08091E100877F8093E3
:1018A000E10082E08093E5011092E1018091E10086
:1018B0008E7F8093E1008091E2008E7F8093E20032
:1018C0008091E20080618093E20042E060E080E08D
:1018D0000E94AF0A8091F00088608093F0000E941F
:1018E0002508FF91EF91BF91AF919F918F917F91CB
:1018F0006F915F914F913F912F910F900FBE0F907D
:101900001F9018951F920F920FB60F9211242F93CC
:101910003F934F935F936F937F938F939F93AF9377
:10192000BF93CF93EF93FF93C091E900CF70809165
:10193000EC001092E9008091F000877F8093F00026
:1019400078940E94BE0C1092E9008091F0008860AB
:101950008093F000C093E900FF91EF91CF91BF9188
:10196000AF919F918F917F916F915F914F913F9137
:101970002F910F900FBE0F901F9018951F93CF932C
:10198000DF93CDB7DEB7AA970FB6F894DEBF0FBED0
:10199000CDBFE6EEF1E08091F100819321E0EE3ED3
:1019A000F207C9F70E9444088091E80083FF1CC138
:1019B0002091E6013091E701832F90E08A30910574
:1019C00008F012C1FC01EA5AFF4F0C948022203823
:1019D00081F0223809F008C18091EA018F7080936C
:1019E000E9008091EB0085FB882780F91092E900DF
:1019F00006C08091E2019091E30191118260909183
:101A0000E800977F9093E8008093F1001092F10036
:101A1000C5C0822F8D7F09F0E7C0222319F0223044
:101A200061F0E2C08091E801813009F0DDC033301F
:101A300009F080E08093E30128C08091E8018111E2
:101A400024C02091EA012F7009F4CEC02093E90050
:101A50008091EB0080FF19C08091EB00333011F4CE
:101A6000806211C080618093EB0081E090E0022EE3
:101A700001C0880F0A94EAF78093EA001092EA0006
:101A80008091EB0088608093EB001092E9008091D8
:101A9000E800877F86C02111A7C01091E8011F7759
:101AA0008091E3008078812B8093E3008091E800AF
:101AB000877F8093E8000E94E40A8091E80080FF1D
:101AC000FCCF8091E30080688093E300112311F044
:101AD00083E001C082E08093E50186C02058223077
:101AE00008F082C08091E8019091E9018C3D23E0EB
:101AF000920779F583E08A838AE289834FB7F89465
:101B0000DE01139620E03EE051E2E32FF0E0509337
:101B10005700E49120FF03C0E295EF703F5FEF7044
:101B20008E2F90E0EA3010F0C79601C0C0968D93DA
:101B30009D932F5F243149F74FBF8091E800877F45
:101B40008093E8006AE270E0CE0101960E94EC0901
:101B500014C0AE014F5F5F4F6091EA010E943409EB
:101B6000009709F441C02091E800277F2093E80006
:101B7000BC0189819A810E944D0A8091E8008B778F
:101B80008093E80031C0203879F58091E800877FA4
:101B90008093E8008091E1018093F1008091E8005A
:101BA0008E778093E8000E94E40A1EC021111CC0B9
:101BB0009091E8019230C0F48091E800877F809393
:101BC000E8009093E1010E94E40A8091E101811113
:101BD00004C08091E30087FF02C084E001C081E07F
:101BE0008093E5010E9430088091E80083FF0AC0DD
:101BF0008091E800877F8093E8008091EB0080620D
:101C00008093EB00AA960FB6F894DEBF0FBECDBF4F
:101C1000DF91CF911F9108950895CF938091E501B1
:101C20008823B1F08091E9008F709091EC0090FFD3
:101C300002C090E801C090E0C92FC82B1092E900C3
:101C40008091E80083FD0E94BE0CCF70C093E90034
:101C5000CF91089590936901809368010895E09170
:101C60006801F0916901309721F00190F081E02D39
:101C7000099480E00895E0916801F091690130973E
:101C800021F00280F381E02D09940895E09168012C
:101C9000F0916901309721F00480F581E02D0994DD
:101CA000089520916601309167018217930771F0C2
:101CB0009093670180936601E0916801F09169015A
:101CC000309721F00680F781E02D09940895209146
:101CD0006401309165018217930771F0909365015B
:101CE00080936401E0916801F0916901309721F0DF
:101CF0000084F185E02D0994089508950C947D0EDB
:101D00000E946F1A0E940B040C94351BCF92DF9235
:101D1000EF92FF920F931F93CF93DF93CDB7DEB770
:101D20002B970FB6F894DEBF0FBECDBF0E942304E1
:101D30003BE6E32E31E0F32E00E010E0C02E802FD2
:101D40000E941005F701D1907F01D826B1F40F5FF2
:101D50001F4F0E30110591F78FEF89838A831B8205
:101D60000E94781A8160782F9D838C8349815A81E3
:101D70006B818D810E94290F41C09091CC0191FF10
:101D800004C08B870E9416058B8520E030E04D2D26
:101D900050E0922FBA01022E02C0759567950A9401
:101DA000E2F760FF25C02E83CF82EE24E394F12C6E
:101DB00002C0EE0CFF1C9A95E2F790E08E219F2165
:101DC00021E0892B09F420E028870E94781A81609D
:101DD000782F9A8789874E815F8168858A850E94DE
:101DE000290FF801E559FE4F80818E25808306C0BA
:101DF0002F5F3F4F2630310561F6A9CF0E94191E93
:101E000010916A010E942F0E1817A1F00E942F0E48
:101E100080936A012B960FB6F894DEBF0FBECDBF3C
:101E2000DF91CF911F910F91FF90EF90DF90CF90B6
:101E30000C9434072B960FB6F894DEBF0FBECDBFBF
:101E4000DF91CF911F910F91FF90EF90DF90CF9096
:101E50000895CF93DF93CDB7DEB72B970FB6F894E5
:101E6000DEBF0FBECDBF4F83588769877A878B87C8
:101E7000DE01119686E0FD0111928A95E9F785E071
:101E8000FE01379601900D928A95E1F749815A81BA
:101E90006B817C818D819E810E945C162B960FB692
:101EA000F894DEBF0FBECDBFDF91CF910895CF93E1
:101EB000C82F882309F4C1C0823859F40E942F0E1C
:101EC00081FDBBC089E30E94F9180E94B31989E320
:101ED0000CC0833879F40E942F0E80FDAEC083E5DC
:101EE0000E94F9180E94B31983E50E943919CF9115
:101EF0000C94B319843859F40E942F0E82FD9DC0B2
:101F000087E40E94F9180E94B31987E4EECF8CEFA2
:101F10008C0F813A48F48C2F0E944E2081118DC085
:101F20008C2F0E94F918E3CF80E28C0F883048F4A0
:101F3000C77081E001C0880FCA95EAF70E947A193C
:101F4000D6CF8BE58C0F833078F4C53A29F0C63AAA
:101F500031F482E890E005C081E890E002C083E8B7
:101F600090E0CF910C94510E88E58C0F833108F0EE
:101F700064C0C83A39F1C93A41F1CA3A49F1CB3A99
:101F800051F1CC3A59F1CD3A61F1C03B69F1CE3A09
:101F900071F1CF3A79F1C13B81F1C23B89F1C33B89
:101FA00091F1C43B99F1C53BA1F1C63BA9F1C73BF7
:101FB000B1F1C83BB9F1C93BC1F1CA3BC9F58AE2ED
:101FC00092E038C082EE90E035C089EE90E032C0F9
:101FD0008AEE90E02FC085EB90E02CC086EB90E07D
:101FE00029C087EB90E026C08CEC90E023C08DECFC
:101FF00090E020C083E891E01DC08AE891E01AC01B
:1020000082E991E017C084E991E014C081E292E096
:1020100011C083E292E00EC084E292E00BC085E240
:1020200092E008C086E292E005C087E292E002C03A
:1020300080E090E0CF910C94670ECF9108958823B3
:1020400009F44BC0823859F40E942F0E81FF45C01D
:1020500089E30E94F9180E94B31989E30CC0833800
:1020600071F40E942F0E80FF38C083E50E94F9189A
:102070000E94B31983E50E9439190C94B31984386E
:1020800059F40E942F0E82FF28C087E40E94F9189D
:102090000E94B31987E4EFCF9CEF980F913A58F361
:1020A00090E2980F983050F4877091E001C0990F3A
:1020B0008A95EAF7892F0E948019DFCF9BE5980F58
:1020C000933020F480E090E00C94510E885A8331D4
:1020D00020F480E090E00C94670E0895882321F0AE
:1020E0000E947A190C94B3190895882321F00E9454
:1020F00080190C94B3190895CF92DF92EF92FF925A
:102100000F931F93CF93DF93CDB7DEB728970FB60A
:10211000F894DEBF0FBECDBF8C0185E0F801DE0173
:10212000119601900D928A95E1F7F8014081318175
:10213000F280258122952F7083819481892B31F043
:102140003F3F31F481E04F3F19F403C081E001C00B
:1021500080E080FDC4C249833A8389819A812F83BC
:102160000E94B7189E8388870E94B6180E9489171C
:102170004E81E42FE295EF70F0E0E05AFF4F2F819F
:1021800068850C948022842F807F142F1F708823F1
:1021900011F01295107FFF2059F0112309F454C259
:1021A000812F68870E948A190E94B31968854CC2E2
:1021B000862F0E941F10112309F491C2812F0E94C3
:1021C000901928960FB6F894DEBF0FBECDBFDF91F1
:1021D000CF911F910F91FF90EF90DF90CF900C94D3
:1021E000B319342F307F842F8F70303211F08295E5
:1021F000807F662319F0613019F12BC0FF20B1F008
:10220000222309F493C1213009F090C128960FB61A
:10221000F894DEBF0FBECDBFDF91CF911F910F911C
:10222000FF90EF90DF90CF900C949A19222319F031
:10223000213009F454C28E830E949D198E8189C178
:10224000FF2021F0223008F04AC270C1211147C29C
:1022500080C1FF2021F0222309F468C1F5C12223A7
:1022600009F477C105C2242F26952695237030E006
:102270002115310521F021303105C9F030C2FF2090
:1022800021F0862F942F937002C080E090E0289672
:102290000FB6F894DEBF0FBECDBFDF91CF911F9177
:1022A0000F91FF90EF90DF90CF900C94510EFF2094
:1022B00021F0862F942F937002C080E090E0289642
:1022C0000FB6F894DEBF0FBECDBFDF91CF911F9147
:1022D0000F91FF90EF90DF90CF900C94670E862FB8
:1022E000FF2019F00E94211D02C00E94891D28961E
:1022F0000FB6F894DEBF0FBECDBFDF91CF911F9117
:102300000F91FF90EF90DF90CF900C940E1E842FD2
:10231000837009F076C0F110E2C1262F2295269530
:102320002770220F220F862F8F70C82ED12CE12C00
:10233000F12C022E04C0CC0CDD1CEE1CFF1C0A94F8
:10234000D2F764FF10C06FE070E080E090E004C05E
:10235000660F771F881F991F2A95D2F76095709591
:102360008095909503C060E070E0CB01242F269506
:1023700026952370422F50E042305105D1F0433072
:10238000510559F16C297D298E299F29413051052C
:1023900041F128960FB6F894DEBF0FBECDBFDF9196
:1023A000CF911F910F91FF90EF90DF90CF900C9401
:1023B000AE176C297D298E299F2928960FB6F8948F
:1023C000DEBF0FBECDBFDF91CF911F910F91FF9068
:1023D000EF90DF90CF900C94C8170E94AE17C70102
:1023E000B60128960FB6F894DEBF0FBECDBFDF91C1
:1023F000CF911F910F91FF90EF90DF90CF900C94B1
:102400009417FF2019F0842F817001C086958823CE
:1024100009F465C1262F229526952770220F220FD9
:10242000862F8F70C82ED12CE12CF12C022E04C0E7
:10243000CC0CDD1CEE1CFF1C0A94D2F764FF10C00C
:102440006FE070E080E090E004C0660F771F881FA7
:10245000991F2A95D2F7609570958095909503C045
:1024600060E070E0CB01242F269526952370422F43
:1024700050E042305105D1F04330510559F16C29FB
:102480007D298E299F294130510541F128960FB6AB
:10249000F894DEBF0FBECDBFDF91CF911F910F919A
:1024A000FF90EF90DF90CF900C9482186C297D29DB
:1024B0008E299F2928960FB6F894DEBF0FBECDBF98
:1024C000DF91CF911F910F91FF90EF90DF90CF9010
:1024D0000C949C180E948218C701B60128960FB66A
:1024E000F894DEBF0FBECDBFDF91CF911F910F914A
:1024F000FF90EF90DF90CF900C946818603FC9F187
:1025000018F4603E50F49BC0623F09F460C008F4C8
:102510004AC0633F09F46FC092C0162F1F70842F0A
:102520008F71FF2099F00E940118812F28960FB615
:10253000F894DEBF0FBECDBFDF91CF911F910F91F9
:10254000FF90EF90DF90CF900C946E100E942218B5
:10255000812F28960FB6F894DEBF0FBECDBFDF9156
:10256000CF911F910F91FF90EF90DF90CF900C943F
:102570007510FF20A1F02111B2C0842F8F71289611
:102580000FB6F894DEBF0FBECDBFDF91CF911F9184
:102590000F91FF90EF90DF90CF900C94471822306E
:1025A00008F09DC0EACFFF20A1F0842F8F712896FC
:1025B0000FB6F894DEBF0FBECDBFDF91CF911F9154
:1025C0000F91FF90EF90DF90CF900C940118FF20B7
:1025D00061F3842F8F7128960FB6F894DEBF0FBE7B
:1025E000CDBFDF91CF911F910F91FF90EF90DF90C2
:1025F000CF900C942218FF2091F0842F8F71289691
:102600000FB6F894DEBF0FBECDBFDF91CF911F9103
:102610000F91FF90EF90DF90CF900C94EC172896DD
:102620000FB6F894DEBF0FBECDBFDF91CF911F91E3
:102630000F91FF90EF90DF90CF900C94E217FF2066
:10264000A1F0222309F4B1CF862F28960FB6F89473
:10265000DEBF0FBECDBFDF91CF911F910F91FF90D5
:10266000EF90DF90CF900C94570F222309F4B1CF55
:10267000862F28960FB6F894DEBF0FBECDBFDF9130
:10268000CF911F910F91FF90EF90DF90CF900C941E
:102690001F104F70C8010E94AB0228960FB6F89425
:1026A000DEBF0FBECDBFDF91CF911F910F91FF9085
:1026B000EF90DF90CF900C9409174F70C8012896C7
:1026C0000FB6F894DEBF0FBECDBFDF91CF911F9143
:1026D0000F91FF90EF90DF90CF900C94D605289645
:1026E0000FB6F894DEBF0FBECDBFDF91CF911F9123
:1026F0000F91FF90EF90DF90CF9008950E9497196F
:102700000E946C190E94B3190E94BA1E0E940E1EEC
:1027100080E090E00E94510E80E090E00C94670E03
:102720000E9487190C947E130E94B718292F2295B6
:102730002F7030E02C3031054CF42A3031056CF428
:10274000225031092230310590F407C02C30310578
:1027500051F02F30310539F00AC0803E10F0803F33
:1027600031F481E0089593FB882780F9089580E093
:102770000895CF93DF9300D000D01F92CDB7DEB77E
:102780000F900F900F900F900F90DF91CF910895C1
:10279000CF93DF9300D000D000D0CDB7DEB7269620
:1027A0000FB6F894DEBF0FBECDBFDF91CF91089575
:1027B0001F93CF93DF93C091790116E080917A0146
:1027C000C81799F0D0E01C9FF0011D9FF00D112457
:1027D000E558FE4F408151816281738184819581EA
:1027E0000E94C8132196C770E9CFDF91CF911F9146
:1027F00008954091AB015091AC016091AD01709191
:10280000AE018091AF019091B0010C94C813CF93A9
:102810008091B00182958F7009F05FC08091AD0109
:10282000882309F45AC020917901A0917A0160911E
:10283000AB017091AC018091AE019091AF0131E09C
:102840006F3F09F030E0B32FC6E02A1709F445C006
:10285000009721F07F3F21F44B2F03C041E001C0DE
:1028600040E030E040FD35C0C29FF001C39FF00D55
:102870001124E558FE4F418174132BC0408164132D
:1028800028C04281411125C043815481481759070E
:1028900010F441505109481B590B483C5105C8F4EC
:1028A0008091B0018F7080618093B00186E0829F3B
:1028B000F001839FF00D1124E058FE4F80818F704E
:1028C000806180838BEA91E00E947C10CF910C9410
:1028D000D8132F5F3F4F2770B8CFCF910895CF9275
:1028E000DF92EF92FF920F931F93CF93DF93CDB7B9
:1028F000DEB762970FB6F894DEBF0FBECDBF8C0176
:1029000085E0F801DE011D9601900D928A95E1F7B0
:10291000D8014C9111965C91119712966C91129777
:102920001396ED90FC9014977091AB01E091AC017F
:102930002091AE013091AF012115310531F0EF3F0B
:1029400031F481E07F3F19F403C081E001C080E0F1
:10295000B82FB170CB2E80FD6CC1D090AD01DD20C1
:1029600009F4F5C0F091B001E216F30638F0C701A2
:10297000821B930B883C910548F09BC020953095B5
:102980002E0D3F1D283C310508F093C08F2F807F0E
:1029900009F052C0E51314C0741312C0D62E611191
:1029A0000FC0FF70F061F093B0010E94F9138BEA41
:1029B00091E00E947C108091B001F80185836CC188
:1029C000EF2831F05F3F31F481E04F3F19F403C04D
:1029D00081E001C080E080FD03C081E0862701C066
:1029E00080E0F82FF170FF2E80FF1CC080917901EC
:1029F00020917A0136E0821709F428C190E0389FCF
:102A0000F001399FF00D1124E558FE4F71815713E5
:102A100006C07081471303C07281671303C001961B
:102A20008770E9CFD62E662309F436C18091B001B4
:102A300081608093B00153C0E51308C0741306C0D1
:102A4000611104C0D8011596FC93AEC04D875E8716
:102A50008D859E856A8B0E9494136A89882329F14B
:102A6000D62E662311F12091B001822F82958F70AE
:102A700090E002970CF460C08091AB019091AC01A2
:102A800098878F831986FB86EA862C87CE01079666
:102A900051C0E51731F14D875E878D859E856A8B24
:102AA0000E9494136A8981112EC0C8010E947C1073
:102AB000A4C08F2F807F69F77E2DF98AE88A8989E3
:102AC0000E94B9138BEA91E00E947C10EBEAF1E0DE
:102AD00086E0DF011D928A95E9F70E94F913D12C57
:102AE000DBC07413D8CF6111D6CFD8011596FC93F3
:102AF000C8010E947C10EBEAF1E086E0DF011D9244
:102B00008A95E9F7C9C0D62E662379F22091B001E3
:102B1000822F82958F7090E0029774F08091AB01C4
:102B20009091AC019A8389831B82FD82EC822E8373
:102B3000CE0101960E947C1086E0F801ABEAB1E07C
:102B400001900D928A95E1F70E9407146FC0E2167A
:102B5000F30628F0C701821B930B9C0104C020954B
:102B600030952E0D3F1D283C310508F052C0D62E61
:102B7000662309F49ACFE5132CC074132AC0809100
:102B8000B00180FD1DC0982F92959F70C9F0D801AB
:102B900015968C9315979F3039F09F5F9295907F93
:102BA0008F70892B15968C93C8010E947C1086E04B
:102BB000F801ABEAB1E001900D928A95E1F736C0D9
:102BC00086E0F801ABEAB1E001900D928A95E1F759
:102BD00063C04D875E878D859E850E9494138823F0
:102BE00079F086E0F801ABEAB1E001900D928A95A8
:102BF000E1F70E9407140E94F913DD24D3944CC01E
:102C00008091B00181608093B001C8010E947C1066
:102C100043C07E2DF98AE88A89890E94B913EBEABC
:102C2000F1E086E0DF011D928A95E9F70E94F91331
:102C300033C0662309F439CF4D875E878D859E8525
:102C40000E949413882309F430CFCBCF4D875E8741
:102C50008D859E850E94B718292F22952F7030E010
:102C6000223031052CF49F7041F0811106C00CC058
:102C7000243031052CF49F7049F4805E883020F0B8
:102C8000C8010E947C10CF2CDC2C06C0D801159600
:102C90009C91907F91F7F8CF8D2D62960FB6F894A6
:102CA000DEBF0FBECDBFDF91CF911F910F91FF907F
:102CB000EF90DF90CF9008951F93CF93DF93CDB720
:102CC000DEB72C970FB6F894DEBF0FBECDBF4F8393
:102CD000588769877A878B879C87CE0107960E94E1
:102CE0006F148823C1F02F8138858A859B85892BB5
:102CF00031F03F3F11F080E003C02F3FE1F781E06A
:102D0000811147C04F81588569857A858B859C855F
:102D10000E94C8133EC086E0FE013796DE01119680
:102D200001900D928A95E1F7FF81E8854A855B85E0
:102D30004115510531F0EF3F31F481E0FF3F19F4C7
:102D400003C081E001C080E080FD23C020917A01B2
:102D500030E0C9010196877099276091790170E090
:102D600086179707F1F1F983EA835D834C8396E038
:102D7000929FD001939FB00D1124A558BE4FFE0124
:102D8000319601900D929A95E1F780937A010E9415
:102D9000D81316E08091790190917A01891779F121
:102DA000189FC001112485589E4F0E946F148823DC
:102DB00031F1E09179011E9FF0011124E558FE4F99
:102DC0004081518162817381848195810E94C81301
:102DD0008091790190E0019687709927809379011D
:102DE000D9CF0E94901310927A0110927901EBEAE8
:102DF000F1E086E0DF011D928A95E9F7CACF2C96B3
:102E00000FB6F894DEBF0FBECDBFDF91CF911F91FB
:102E10000895EF92FF920F931F93CF93DF93FC01DE
:102E2000009709F46FC0F12CEE24E394EF01219692
:102E30008491843740F4843008F055C0813081F0AB
:102E4000823021F15FC0853709F447C0C0F19CE7AB
:102E5000980F903708F056C08F770E941F1045C01A
:102E60008F010E5F1F4FFE01849190E2980F983002
:102E700050F48770FE2D01C0FF0F8A95EAF78F2F5F
:102E80000E948A1915C00E94570F14C08F010E5F4F
:102E90001F4FFE01849190E2980F983068F487707C
:102EA000FE2D01C0FF0F8A95EAF78F2F0E9490191F
:102EB0000E94B319E80119C00E941F10FBCFCF0177
:102EC0000296FE01C491CC2361F0EFE9FFE0319757
:102ED000F1F700C00000C150F6CFCF010296FE010D
:102EE000F490EC0102C00E94570F8F2D882341F00F
:102EF000EFE9FFE03197F1F700C000008150F6CF15
:102F0000FE0194CFDF91CF911F910F91FF90EF9031
:102F1000089508956093B5017093B6018093B70149
:102F20009093B8010C947E130F931F930091B501F9
:102F30001091B6012091B7013091B801062B172BE3
:102F4000282B392B0093B5011093B6012093B701BC
:102F50003093B8011F910F910C947E130F931F9320
:102F60000091B5011091B6012091B7013091B801DF
:102F700006231723282339230093B5011093B601A4
:102F80002093B7013093B8011F910F910C947E13D9
:102F90000F931F930091B5011091B6012091B701D5
:102FA0003091B80106271727282739270093B50144
:102FB0001093B6012093B7013093B8011F910F9180
:102FC0000C947E131092B1011092B2011092B301D1
:102FD0001092B4010C947E1341E050E060E070E088
:102FE00004C0440F551F661F771F8A95D2F7409380
:102FF000B1015093B2016093B3017093B4010C948A
:103000007E1341E050E060E070E004C0440F551FC3
:10301000661F771F8A95D2F78091B1019091B20116
:10302000A091B301B091B401842B952BA62BB72BA3
:103030008093B1019093B201A093B301B093B40116
:103040000C947E1341E050E060E070E004C0440F57
:10305000551F661F771F8A95D2F74095509560954A
:1030600070958091B1019091B201A091B301B0919E
:10307000B40184239523A623B7238093B1019093B1
:10308000B201A093B301B093B4010C947E1341E05C
:1030900050E060E070E004C0440F551F661F771FCA
:1030A0008A95D2F78091B1019091B201A091B301BC
:1030B000B091B40184279527A627B7278093B10143
:1030C0009093B201A093B301B093B4010C947E131A
:1030D0000F931F930091B1011091B2012091B301A0
:1030E0003091B401062B172B282B392B0093B101FB
:1030F0001093B2012093B3013093B4011F910F914B
:103100000C947E130F931F930091B1011091B201A3
:103110002091B3013091B4010623172328233923CA
:103120000093B1011093B2012093B3013093B40125
:103130001F910F910C947E130F931F930091B10177
:103140001091B2012091B3013091B40106271727E5
:10315000282739270093B1011093B2012093B301BE
:103160003093B4011F910F910C947E130895CF9268
:10317000DF92EF92FF920F931F93CF93DF93EC01B7
:10318000C090B501D090B601E090B701F090B801C1
:103190008091B1019091B201A091B301B091B401BD
:1031A000C82AD92AEA2AFB2A0FE110E0B701A601B2
:1031B000002E04C076956795579547950A94D2F7E7
:1031C00040FF07C0BE01802F0E94F90581309105A4
:1031D00039F40150110950F7BE0180E00E94F90551
:1031E000DF91CF911F910F91FF90EF90DF90CF90E3
:1031F000089590910C019923D9F090910D01992394
:10320000B9F0982F9695969596959F3088F5E09110
:103210000E01F0910F01E90FF11D877021E030E000
:1032200001C0220F8A95EAF78181822B818308955C
:1032300040910E0150910F0120E030E09FEFFA0124
:10324000E20FF31F6281681799F09F3F19F4611133
:1032500001C0922F2F5F3F4F2E30310581F79F3FE6
:1032600039F0FA01E90FF11D97FDFA95828308956F
:10327000089590910C019923E1F090910D0199230B
:10328000C1F0982F9695969596959F3020F5E091F0
:103290000E01F0910F01E90FF11D877021E030E080
:1032A00001C0220F8A95EAF7209581812823218386
:1032B000089540910E0150910F0120E030E0FA0195
:1032C000E20FF31F9281981301C012822F5F3F4FCC
:1032D0002E303105A1F7089581E090E0E0910E01D4
:1032E000F0910F01E80FF91F1082019680319105CE
:1032F000A9F708959091CB01982B9093CB01089555
:1033000080959091CB0198239093CB0108951092D2
:10331000CB0108959091CA01982B9093CA0108950A
:1033200080959091CA0198239093CA0108951092B4
:10333000CA0108958093B90108951092B9010895C2
:1033400040910E0150910F0120E030E080E0FA0141
:10335000E20FF31F918191118F5F2F5F3F4F2F304D
:103360003105A9F70895E0910E01F0910F018091C8
:10337000CB018083E0910E01F0910F01808190914B
:10338000CA01892B80839091B901992361F0E09162
:103390000E01F0910F018081892B80830E94A0197A
:1033A00081111092B90180910E0190910F010C943E
:1033B0003B0ECF92DF92EF92FF920F931F936C011F
:1033C000EE24FF24C114D104E104F10421F46B01C3
:1033D0007C0180E001C080E133272F2D1E2D0D2DB3
:1033E000011511052105310519F0885F6801790182
:1033F00097018601A4E03695279517950795AA951C
:10340000D1F7011511052105310519F08C5F68010F
:10341000790197018601F2E0369527951795079572
:10342000FA95D1F7011511052105310519F08E5FC7
:1034300068017901B701A60176956795579547957B
:10344000452B462B472B09F08F5F1F910F91FF9063
:10345000EF90DF90CF9008958091E501843009F1DD
:103460001092CD0120E488E190E00FB6F894A89581
:10347000809360000FBE2093600083B7817F8460DB
:1034800083BF83B7816083BF7894889583B78E7F2D
:1034900083BF88E10FB6F8948093600010926000BB
:1034A0000FBE089508950895CF930E94521A0E9466
:1034B00023040E94531AC0E08C2F0E941005811132
:1034C00005C0CF5FCE30C1F780E001C081E0CF9171
:1034D00008950E9490130E942F0E0C94340782E0EE
:1034E00084BD93E095BD9AEF97BD80936E000895DB
:1034F0002FB7F8948091CE019091CF01A091D00187
:10350000B091D1012FBF0895CF92DF92EF92FF9239
:103510000F931F932FB7F8944091CE015091CF0194
:103520006091D0017091D1012FBF6A017B01EE241F
:10353000FF248C0120E030E0C016D106E206F3063D
:1035400010F441505109481B590BCA011F910F91AA
:10355000FF90EF90DF90CF9008951F920F920FB6DB
:103560000F9211248F939F93AF93BF938091CE01BD
:103570009091CF01A091D001B091D1010196A11DF0
:10358000B11D8093CE019093CF01A093D001B09351
:10359000D101BF91AF919F918F910F900FBE0F906E
:1035A0001F9018950E94350BF8942FEF87EA91E64B
:1035B000215080409040E1F700C0000087E090EB90
:1035C000DC018093EE019093EF01A093F001B093A2
:1035D000F1012CE088E190E00FB6F894A895809373
:1035E00060000FBE20936000FFCFEF92FF920F9319
:1035F0001F93CF93DF93E82EF12C8F2D0E9410059F
:10360000C0E0D0E0082F10E098010C2E02C03595E4
:1036100027950A94E2F720FD05C02196C630D10512
:1036200099F709C06C2F7F2D80E00E94D705E81222
:10363000F4CF81E005C0F3948EE0F812DECF80E095
:10364000DF91CF911F910F91FF90EF900895CF934D
:10365000C82F8CE20E94F51A882321F08C2FCF917D
:103660000C94F51A80E0CF910895CF930E947A1CB4
:10367000811102C00E94601CC5E6C15049F00E9441
:1036800023048FE39CE90197F1F700C00000F5CF18
:1036900089E20E94271B811111C18AE20E94271B27
:1036A00081110E94601C85E00E94271B81110E94ED
:1036B000D21A0E94851C8093CC0187E00E94271BB0
:1036C000882399F18BE10E94271B882351F0909168
:1036D000CC0191FB882780F921E0822780FB91F9BA
:1036E00022C08EE00E94271B882351F09091CC01CC
:1036F00092FB882780F921E0822780FB92F913C092
:1037000080E10E94271B9091CC01882341F093FB1C
:10371000882780F921E0822780FB93F904C0892F54
:10372000809580FB90F99093CC018091CC010E9410
:10373000891C0E94971C8093DF0180EE0E94271B4A
:10374000882341F08091DF01982F909590FB80F9BC
:103750008093DF0189E30E94271B882359F0909111
:10376000DF0191FB882780F921E0822780FB91F916
:103770009093DF0182EE0E94271B882359F09091DD
:10378000DF0192FB882780F921E0822780FB92F9F4
:103790009093DF0186EE0E94271B882359F09091B9
:1037A000DF0193FB882780F921E0822780FB93F9D2
:1037B0009093DF0183EE0E94271B882359F090919C
:1037C000DF0194FB882780F921E0822780FB94F9B0
:1037D0009093DF0185E30E94271B882359F0909185
:1037E000DF0195FB882780F921E0822780FB95F98E
:1037F0009093DF0181E30E94271B882359F0909169
:10380000DF0196FB882780F921E0822780FB96F96B
:103810009093DF0181E10E94271B882359F090914A
:10382000DF0197FB882780F921E0822780FB97F949
:103830009093DF018091DF010E949B1C8091DF014A
:1038400087FB882780F980930D0187E20E94271B60
:10385000C82F8EE10E94271B8111C2608FE10E9458
:10386000271B8111C46080E20E94271B8111C86060
:1038700081E20E94271B8111C06182E20E94271B06
:103880008111C06283E20E94271B8111C06484E21F
:103890000E94271B882311F0C06802C0CC2329F0A6
:1038A0008C2F0E94921C6C2F03C00E948E1C682FCC
:1038B00070E080E090E0CF910C948A17CF9108954A
:1038C0006DEE7EEF80E090E00E94B62260E082E044
:1038D00090E00E94A82260E083E090E00E94A8228D
:1038E00060E084E090E00E94A82260E085E090E043
:1038F0000C94A82280E090E00E94A22221E08D3E5C
:103900009E4F09F020E0822F089582E090E00C9411
:103910009A22682F82E090E00C94A82283E090E045
:103920000C949A22682F83E090E00C94A82284E003
:1039300090E00C949A22682F84E090E00C94A822E6
:103940008091D40180FF0BC06091130185E0689FD6
:10395000B001112475956795759567952AC081FF0B
:1039600009C06091130185E0689FB001112475952D
:1039700067951FC082FF07C06091130185E0689FB3
:10398000B001112416C04091D5014423C9F06091C3
:103990001201461788F72091130185E0289F9001B6
:1039A0001124429FC001439F900D112470E00E949A
:1039B0006C226038710540F46115710539F002C060
:1039C00065E070E0862F08958FE7089581E00895FF
:1039D0008091D40180FF08C06091110170E075955D
:1039E00067957595679521C081FF06C060911101AB
:1039F00070E07595679519C082FF04C06091110150
:103A000070E010C08091D5018823C1F06091100151
:103A10008617A0F790911101989FC001112470E0C2
:103A20000E946C226038710528F46115710521F03F
:103A3000862F08958FE7089581E0089561E070E092
:103A4000F4CF803F21F40E94A01C819504C0813FE7
:103A500029F40E94A01C8093D8010895823F21F48C
:103A60000E94A01C819504C0833F29F40E94A01CE1
:103A70008093D7010895893F19F40E94E81C05C07E
:103A80008A3F31F40E94E81C81958093D901089502
:103A90008B3F21F40E94E81C819504C08C3F29F4DF
:103AA0000E94E81C8093DA010895843F21F48091FC
:103AB000D601816017C0853F21F48091D6018260D4
:103AC00011C0863F21F48091D60184600BC0873FEE
:103AD00021F48091D601886005C0883F31F480913F
:103AE000D60180618093D60108958D3F21F48091A5
:103AF000D40181600BC08E3F21F48091D40182609B
:103B000005C08F3F29F48091D40184608093D40153
:103B10000895803F39F48091D80187FF6CC01092DE
:103B2000D80169C0813F29F48091D8011816BCF3EF
:103B300062C09091D701823F29F497FF5CC0109238
:103B4000D70159C0833F19F41916CCF354C0893FEB
:103B500041F48091D90118160CF04DC01092D90192
:103B60004AC08A3F29F48091D90187FF44C0F6CF2B
:103B70008B3F39F48091DA0187FF3DC01092DA0162
:103B80003AC08C3F29F48091DA011816BCF333C097
:103B9000843F21F48091D6018E7F17C0853F21F4A8
:103BA0008091D6018D7F11C0863F21F48091D6018E
:103BB0008B7F0BC0873F21F48091D601877F05C0A2
:103BC000883F31F48091D6018F7E8093D60113C057
:103BD0008D3F21F48091D4018E7F0BC08E3F21F464
:103BE0008091D4018D7F05C08F3F29F48091D4014D
:103BF0008B7F8093D4018091D70181110EC0809179
:103C0000D80181110AC08091D901811106C080912B
:103C1000DA01811102C01092D501089586ED91E07C
:103C20000E94460E0E94781A9093D3018093D2018D
:103C300008951F93CF93DF938091D2019091D30188
:103C40000E94841A4091D501442321F0209114014F
:103C500030E006C0209115015AE0259F9001112403
:103C60008217930708F482C08091D7011091D80180
:103C7000D091D901C091DA01811107C0111105C09D
:103C8000D11103C0CC2309F471C04F3F19F04F5F2D
:103C90004093D501181624F40E94A01C8093D701EC
:103CA0008091D70187FF05C00E94A01C8195809359
:103CB000D701111624F40E94A01C8093D801809192
:103CC000D80187FF05C00E94A01C81958093D80170
:103CD0006091D701662339F11091D801112319F1B0
:103CE000772767FD7095872F972F0E947D2123E30B
:103CF00033E343E35FE30E94E1210E944A216093A2
:103D0000D701612F772767FD7095872F972F0E9426
:103D10007D2123E333E343E35FE30E94E1210E943B
:103D20004A216093D8011D1624F40E94E81C809358
:103D3000D9018091D90187FF05C00E94E81C8195B7
:103D40008093D9011C1624F40E94E81C8093DA01A8
:103D50008091DA0187FF05C00E94E81C819580935D
:103D6000DA01DF91CF911F910C940E1EDF91CF915C
:103D70001F910895E6EDF1E085E0DF011D928A953F
:103D8000E9F71092D5011092D4010895833081F1A2
:103D900028F4813059F08230D1F00895853009F44B
:103DA00049C0B8F1863009F456C008952091150134
:103DB000862F90E0820F911D8F3F910520F4620FB6
:103DC0006093150108958FEF809315010895209158
:103DD0001401862F90E0820F911D8F3F910520F4F2
:103DE000620F6093140108958FEF8093140108957A
:103DF00020911301862F90E0820F911D8F3F910536
:103E000020F4620F6093130108958FEF80931301E4
:103E1000089520911201862F90E0820F911D8F3F0F
:103E2000910520F4620F6093120108958FEF809343
:103E30001201089520911101862F90E0820F911DAB
:103E40008F3F910520F4620F6093110108958FEF69
:103E500080931101089520911001862F90E0820F28
:103E6000911D8F3F910520F4620F6093100108951A
:103E70008FEF809310010895833011F128F4813081
:103E800049F0823091F00895853081F120F186303B
:103E9000C1F1089580911501681720F4861B809365
:103EA0001501089510921501089580911401681765
:103EB00020F4861B80931401089510921401089534
:103EC00080911301681720F4861B809313010895D5
:103ED00010921301089580911201681720F4861B37
:103EE000809312010895109212010895809111019A
:103EF000681720F4861B8093110108951092110118
:103F0000089580911001681720F4861B809310019A
:103F100008951092100108958D3109F442C020F5E2
:103F20008E3009F479C070F4873009F45EC020F453
:103F3000863009F442C033C08830D1F18B3009F4A7
:103F4000A7C02DC0863109F4A3C038F4803109F42C
:103F50006DC0813109F47BC022C0893109F498C059
:103F60008B3109F44FC01BC0853309F479C048F484
:103F7000873209F475C008F478C0893209F470C03A
:103F80000EC0833438F48A3308F071C0883309F4E2
:103F90007FC005C0833409F463C08834C1F080E079
:103FA00008950E9404210E942F0E0E94340770C0C1
:103FB0000E94851C0E94971C6BC08091CC01817F60
:103FC0008E7F8093CC0181E08093DC0108950E9474
:103FD00090132FEF83ED90E3215080409040E1F764
:103FE00000C000000E94D21A53C09091CC01892FCA
:103FF000817090FF03C0917F9E7F26C09160909357
:10400000CC0146C09091CC0191FB882780F921E03A
:10401000822780FB91F913C09091CC0192FB8827F5
:1040200080F921E0822780FB92F909C09091CC01B0
:1040300093FB882780F921E0822780FB93F99093F6
:10404000CC01882329F191609093CC0108950E94BE
:10405000901380910D0191E0892780930D0118C084
:1040600061E070E080E090E00FC023EE01C027EC3B
:10407000280F61E070E080E090E004C0660F771FD9
:10408000881F991F2A95D2F70E948A170E949013C1
:1040900081E0089580E0089580E00895CF93C82FCF
:1040A0008091DC01813079F018F08230D1F184C048
:1040B000A0910E01B0910F018C91813169F0823293
:1040C00009F07CC009C0A0910E01B0910F018C9144
:1040D000813111F0823249F48C2F0E944A208111E3
:1040E0001DC08C2F0E948C1F1AC08C2F0E944C2048
:1040F000811114C0C43179F048F4CB3079F0C0316B
:1041000009F060C082E08093DC0108C0C93219F078
:10411000C83321F057C01092DC0154C081E0817097
:1041200053C0C93289F118F5C43171F1A8F4C73010
:1041300009F046C08AE08093150194E19093140140
:1041400093E0909313018093120188E08093110112
:1041500088E28093100134C0CE51C63088F5EC2F30
:10416000F0E0E65DFE4F80818093DB0129C0CE3414
:10417000E9F020F4CB3421F56AE013C0C13579F0C1
:10418000C235F1F461E00DC08091DB01882319F0A4
:104190001092DB0115C081E08093DC0115C061E065
:1041A00006C08091DB010E94C61E0AC06AE08091B1
:1041B000DB010E943C1F04C01092DC0180E004C0BF
:1041C00081E002C080E0ABCFCF910895E1E8F0E05C
:1041D0008081886080838081816080838FB7F8943C
:1041E00093E09093890090ED909388008FBF08959D
:1041F000EFE6F0E08081826080830895EFE6F0E0F2
:1042000080818D7F80830895EFE6F0E0808192E0E9
:104210008927808308951F920F920FB60F92112461
:104220002F933F934F935F936F937F938F939F93BE
:10423000AF93BF93EF93FF938091DD019091DE01E7
:1042400001969093DE018093DD01811103C082E02D
:104250000E943407E091DE01E695E695F0E0E6572E
:10426000FB4FE4918091DD018E1303C080E00E943A
:104270003407FF91EF91BF91AF919F918F917F9103
:104280006F915F914F913F912F910F900FBE0F90C3
:104290001F90189504D06894B1118DC0089570D006
:1042A00088F09F5790F0B92F9927B751A0F0D1F01F
:1042B000660F771F881F991F1AF0BA95C9F712C0A9
:1042C000B13081F077D0B1E0089574C0672F782FB6
:1042D0008827B85F39F0B93FCCF386957795679515
:1042E000B395D9F73EF490958095709561957F4F81
:1042F0008F4F9F4F0895E89409C097FB3EF4909527
:104300008095709561957F4F8F4F9F4F9923A9F0AE
:10431000F92F96E9BB279395F6958795779567953D
:10432000B795F111F8CFFAF4BB0F11F460FF1BC081
:104330006F5F7F4F8F4F9F4F16C0882311F096E914
:1043400011C0772321F09EE8872F762F05C06623C2
:1043500071F096E8862F70E060E02AF09A95660F7B
:10436000771F881FDAF7880F9695879597F9089534
:1043700057FD9058440F551F59F05F3F71F0479516
:10438000880F97FB991F61F09F3F79F087950895FB
:10439000121613061406551FF2CF4695F1DF08C01A
:1043A000161617061806991FF1CF86957105610537
:1043B00008940895E894BB2766277727CB0197F9DF
:1043C00008950BD078C069D028F06ED018F09523EE
:1043D00009F05AC05FC01124EECFCADFA0F3959F49
:1043E000D1F3950F50E0551F629FF001729FBB27DC
:1043F000F00DB11D639FAA27F00DB11DAA1F649F88
:104400006627B00DA11D661F829F2227B00DA11D3A
:10441000621F739FB00DA11D621F839FA00D611DC0
:10442000221F749F3327A00D611D231F849F600DE1
:10443000211D822F762F6A2F11249F5750408AF01A
:10444000E1F088234AF0EE0FFF1FBB1F661F771FA6
:10445000881F91505040A9F79E3F510570F014C03D
:10446000AACF5F3FECF3983EDCF38695779567958E
:10447000B795F795E7959F5FC1F7FE2B880F911DC4
:104480009695879597F9089597F99F6780E870E06A
:1044900060E008959FEF80EC089500240A941616BA
:1044A000170618060906089500240A941216130622
:1044B000140605060895092E0394000C11F48823B0
:1044C00052F0BB0F40F4BF2B11F460FF04C06F5FCC
:1044D0007F4F8F4F9F4F089597FB072E16F4009440
:1044E00007D077FD09D00E94862207FC05D03EF454
:1044F000909581959F4F0895709561957F4F089590
:10450000EE0FFF1F0590F491E02D0994AA1BBB1B31
:1045100051E107C0AA1FBB1FA617B70710F0A61BC3
:10452000B70B881F991F5A95A9F780959095BC01E4
:10453000CD010895F999FECF92BD81BDF89A9927D2
:1045400080B50895A8E1B0E042E050E00C94BD22AF
:10455000262FF999FECF1FBA92BD81BD20BD0FB69F
:10456000F894FA9AF99A0FBE019608950E94A8222B
:10457000272F0C94A922DC01CB01FC01F999FECF75
:1045800006C0F2BDE1BDF89A319600B40D924150DB
:0A4590005040B8F70895F894FFCFEB
:10459A0020023607C307A0076C0739070101BA01D1
:1045AA0028080A03140A3F4D36394B04FE03C80390
:1045BA008F0322033B0354036D0301020304050620
:0445CA0007080900D5
:00000001FF
